:1000000020C03AC039C038C037C036C035C034C04F
:1000100033C048C731C030C02FC02EC02DC02CC047
:100020002BC02AC029C001020008200400000010D3
:1000300080401E0E1A2C32301224170713253B392C
:100040001B2D11241FBECFE5D4E0DEBFCDBF10E0D5
:10005000A0E6B0E0E0EBFAE102C005900D92A03618
:10006000B107D9F711E0A0E6B0E001C01D92A033BE
:10007000B107E1F774DA1BCDC3CF9FBB8EBBE09A0B
:100080008DB3861719F06DBBE29AE19A0895DC01F1
:10009000FC01359695E082918FB9779BFECF915008
:1000A000D1F7C19AFD011582C1980895DC014F7303
:1000B000FC01643020F033966450623029F16130E5
:1000C00061F0613028F06230C1F0633051F523C037
:1000D0008081807C842B808324C080818F73942FC7
:1000E0009295990F990F907C982B90838181807FB6
:1000F00046954695842B818314C082818C7F942FF2
:1001000092959F70892B828381818F704295407F69
:10011000482B418306C082818370440F440F482BD3
:10012000428381E0FD0185830895E82F772763FDF1
:10013000EA5F86B323B330B3482F41708695982F7A
:100140009270492B2470422B869586958871307E5B
:10015000832B482B64FD4095FF27EA5DFF4FE49118
:100160004E23842F992708958056904025E0959539
:1001700087952A95E1F7089520E630E0F90180851A
:100180008D7F8087205E3F4FB09681E02032380718
:10019000B1F7089520E630E0E2E6F0E08081918159
:1001A000B096205E3F4F41E020323407B9F7089502
:1001B0001F93CF93DF93DC01EC91EC0188858E2BAC
:1001C00084FD02C01FE306C0E295EF70FF27EE5CDE
:1001D000FF4F1491CD01C8DF412F682F81E391E0DB
:1001E00065DFDF91CF911F910895FC018FEF868F1E
:1001F000908190619083808580FD61956295660F06
:10020000607E960F9083CF01D3DF0895CF92DF9267
:10021000EF92FF921F936B017C01122FBA01660FC0
:10022000771F56FF04C09B012250304003C09B0142
:100230002E5F3F4F882777FD8095982F442737FD05
:100240004095542F15DC05C0660F771F881F991F36
:10025000110F1034CCF320E030E0C616D706E806C4
:10026000F90614F421E030E0C9011F91FF90EF90EE
:10027000DF90CF900895FC01828193810097B9F0BF
:100280002481358146815781AA2797FDA095BA2FF1
:10029000820F931FA41FB51F632F691B848395834F
:1002A000A683B783662319F06195CF019EDF089579
:1002B000CF93DF93C0E6D0E0CE01DDDFA09681E0F2
:1002C000C032D807C9F7DF91CF9108951F93CF931C
:1002D000DF93EC011B8D48DFAC01212F332722FD7A
:1002E00007C08F8587FD09C021FF09C088E0182756
:1002F000612F842F1ADF992704C020FDF9CF8FEFDB
:1003000090E0DF91CF911F910895FC0120E030E053
:1003100080819181A281B38182509040A040B048F9
:100320008D5F9F4FAF4FBF4F10F421E030E0C90108
:1003300008951F93FC01138D10FF06C015DF612F78
:10034000F4DE282F33271CC08085992785FF03C042
:1003500020E030E015C081FD02C060E00FC060E029
:10036000248135814681578180899189A289B38909
:10037000281739074A075B070CF461E0262F33275B
:10038000C9011F9108951F93FC01838D81FF09C04E
:1003900018E01827CF01E8DE612FC7DE282F3327AA
:1003A0001CC08085992785FF03C020E030E015C080
:1003B00081FD02C060E00FC060E02481358146818C
:1003C000578184899589A689B78982179307A407DD
:1003D000B5070CF461E0262F3327C9011F9108955A
:1003E000FC0122853385808183FF02C028E030E054
:1003F00060FE08C080913701909138018217930701
:100400000CF49C01C9010895FC01808182FF0BC09E
:1004100082819381813491051CF080858D7F808756
:100420001382128214828081846080830895CF9326
:10043000DF93C0E6D0E0CE01E7DFA09681E0C032D6
:10044000D807C9F7DF91CF9108950F931F93CF93EA
:10045000DF93EB01042F122F87DE9C01E19918C076
:1004600080E390E0A901489F9001499F300D589F7B
:10047000300D1124285F3F4F200F311DFE013FBB7F
:100480002EBBE09A2F5F3F4F8DB381931150B9F788
:10049000DF91CF911F910F910895EF92FF920F93EB
:1004A0001F93CF93DF93EC01EC80FD800E811F81C1
:1004B000BC016C5F7F4F24E048E0C7DFBE01605F96
:1004C0007F4F28E04CE0CE01C0DF888587FF05C064
:1004D00080E090E0A0E0B0E008C08C819D81AE811A
:1004E000BF818E199F09A00BB10B8C879D87AE87AA
:1004F000BF87DF91CF911F910F91FF90EF900895EB
:10050000FC01808581FF37C01482208931894289AE
:100510005389DA01C90182509040A040B0488D5FF4
:100520009F4FAF4FBF4F60F484819581A681B78103
:10053000281B390B4A0B5B0B208B318B428B538B67
:100540002489358946895789DA01C901825090404A
:10055000A040B0488D5F9F4FAF4FBF4F60F4848184
:100560009581A681B781281B390B4A0B5B0B248B25
:10057000358B468B578B80858260808714821582ED
:10058000168217820895CF93DF93C0E6D0E0CE01A4
:10059000B7DFA09681E0C032D807C9F7DF91CF91CD
:1005A0000895FC018085992783FF03C0CF0175DF83
:1005B000089582FF02C081E001C08FEF87878081AC
:1005C000826080830895CF93DF93C0E6D0E0CE01B0
:1005D000E8DFA09681E0C032D807C9F7DF91CF915C
:1005E0000895EF92FF921F93CF93DF93CDB7DEB7BD
:1005F00021970FB6F894DEBF0FBECDBF7C01FC0182
:100600001185198321E045E0BE016F5F7F4F1DDF3B
:100610008981112339F0882319F0811708F4182FE4
:1006200080E406C0182F8823D9F780E403C086959C
:100630001817E8F3F701818721960FB6F894DEBF0B
:100640000FBECDBFDF91CF911F91FF90EF90089526
:10065000FC018081992783709070892B81F08185BE
:1006600067FD09C0992787FD9095880F991F81879D
:10067000CF01B7DF0895859519F081870895678FB9
:1006800008950F931F93CF93DF93CDB7DEB72297D3
:100690000FB6F894DEBF0FBECDBF8C0180E091E0B5
:1006A0009A83898322E046E0BE016F5F7F4FC801D5
:1006B000CCDE89819A81009721F08F3F910519F056
:1006C00014F080E091E0F801228533852115310591
:1006D00019F08217930718F4F801938782872296FE
:1006E0000FB6F894DEBF0FBECDBFDF91CF911F9143
:1006F0000F9108951F93CF93DF93EC01162F8881FC
:10070000992783709070892B91F0262F332727FD2E
:1007100030958A859B85280F391F2115310559F1A0
:100720003B872A8716163CF5CE01ABDF24C067FF56
:1007300005C0CE01FEDD882329F01DC0CE0123DED9
:100740008823C9F4212F332727FD3095322F222704
:10075000442737FD4095542F8C819D81AE81BF8108
:10076000820F931FA41FB51F8C839D83AE83BF830D
:10077000612FCE013ADDDF91CF911F9108950F9344
:100780001F938C01BC016C5F7F4F2AE140E05DDE6E
:10079000C80127DFC80175DF1F910F910895CF931E
:1007A000DF93C0E6D0E0CE01EADFA09681E0C03260
:1007B000D807C9F7DF91CF910895EF92FF920F9379
:1007C0001F93FC01E088F188028913892489358907
:1007D000468957892E193F09400B510B203080E183
:1007E000380780E0480780E05807F4F0848195815D
:1007F000A681B7818E199F09A00BB10B821B930BA9
:10080000A40BB50B0FB602FEF9CF820F931FA41FE6
:10081000B51F0FB600FEF9CF8E0D9F1DA01FB11F93
:1008200084839583A683B7831F910F91FF90EF90E8
:1008300008959F92AF92BF92CF92DF92EF92FF9274
:100840000F931F93CF93DF93EC01B880AF8C0B2DE8
:100850001127C80183709070892BA1F0F984FA0CDC
:10086000FF8E00FD07C001FF05C0CE012FDD8823EC
:1008700011F076C180E002FD73C12FE32F150CF457
:100880006FC190C180E0CA80DB8098849801247099
:10089000307002FD44C001FF42C000FD40C0AF8483
:1008A0008F3F01F52C893D894E895F898889998917
:1008B000AA89BB89A7FC09C02C873D874E875F8723
:1008C0008C839D83AE83BF8308C08C879D87AE8752
:1008D000BF872C833D834E835F8331E0B32A8DEF46
:1008E0009822C8C0882379F003FFC2C095EFB922CF
:1008F000CE01D3DD22E0922A14F431E0B32AAA24F7
:10090000CC24DD24B7C08A2D992787FD90958C0DC6
:100910009D1D892B09F0AEC088E0B82AABC0C11478
:10092000D10409F475C0D7FE37C0232B29F4CE01BA
:1009300000DD882309F416C194E0B92AD6C095FEDB
:100940000CC08C859D85AE85BF8581509040A040B0
:10095000B04819F4CE0131DF58C0EC80FD800E8123
:100960001F818C859D85AE85BF85E81AF90A0A0B23
:100970001B0B2985A601C801B70148DC882329F58E
:100980000894C108D1082985A601C801B7013EDC39
:10099000882309F46FC019C0232B29F4CE01F3DC9E
:1009A000882309F4E2C034E0B32AFFEFAF2EA5C0DC
:1009B00095FE0EC08C859D85AE85BF858F5F9F4F50
:1009C000AF4FBF4729F4CE01F8DEE1E0AE2E52C0B2
:1009D000EC84FD840E851F858C819D81AE81BF8155
:1009E000E81AF90A0A0B1B0B2985A601C801B701F1
:1009F0000DDC882351F40894C11CD11C2985A60163
:100A0000C801B70103DC8823A9F17FEFA72E32C00C
:100A1000232B11F034EFB322B0FE1EC02C853D8590
:100A20004E855F858C819D81AE81BF8128173907F6
:100A30004A075B073CF4CE017CDC882359F46FEF56
:100A4000A62E98C00FB601FC05C0CE019CDC882301
:100A500009F48EC08EEFB82293EFB922AA2051F488
:100A60008E8D882339F081508E8F882319F485C0AC
:100A70008EEFA826862D992780FF23C082FF08C00D
:100A800020E0C03CD207E8F4888581FD7DC019C014
:100A900030E0C03CD30708F077C013C0CE0149DC7A
:100AA000882309F476C051E0A52E0BC0CE016BDC83
:100AB000882309F471C04FEFA42E03C03FEFC32E6B
:100AC000D32ECE018DDC8C159D051CF42FEFA22EAC
:100AD00006C0C816D90619F41A140CF4AA24909565
:100AE00081959F4FC816D9061CF481E0A82E05C039
:100AF000C816D90611F4A7FCAA248A2D992787FDC8
:100B000090958C0D9D1D2A81382F321B232F3985FE
:100B1000239F202D112429839B838A83892B91F481
:100B20008B2D992781FF0EC080FF0CC084EFB82267
:100B3000CE01B3DC92E0992AB2FC04C097FE02C059
:100B400021E0B22AB8828B2D992783709070892B6F
:100B500021F08F8D80548F8F01C01F8E988622C008
:100B6000AA2491CE00FDEBCE85CF00FD21CF82CF10
:100B700001E0A02E33EFB3227DCF8FEEB822B882F2
:100B8000CE0116DB1C8276CF1C141D040CF48BCF17
:100B900085CFD7FE8BCF8FCF61FC90CF11E0C12ED8
:100BA000D12C8FCFDF91CF911F910F91FF90EF90BC
:100BB000DF90CF90BF90AF909F90089580913001CB
:100BC00081BFE0E0FEE009944091350142954F700D
:100BD000882311F4440F440F437F161614F4446025
:100BE00002C067FD4860882311F44695469566E08B
:100BF00081E391E05BDA08951F93182F60FE18C01F
:100C00002091370130913801862F992787FD9095E3
:100C1000280F391F2115310509F446C081E0213024
:100C200038070CF041C030933801209337013CC0A5
:100C3000882319F0E8E2F3E002C0EAE7F3E083E09A
:100C40003816F1F0831530F081E0381691F08315F5
:100C5000A0F00CC085E03816C9F03816A0F086E088
:100C60003816B9F087E03816F9F415C080EC90E03A
:100C700002C080EE90E0099517C080E091E0FBCFC4
:100C800080E690E0F8CF80E890E0F5CF80EA90E051
:100C9000F2CF80E001C081E097DF112311F080E006
:100CA00001C088E780932F011F91089580912F0143
:100CB000882351F0815080932F01882329F440E04C
:100CC00066E081E391E0F2D9089560FC6A94AFDBBD
:100CD00040E066E081E391E0E9D908955D9B15C0AD
:100CE00088E0681619F485E58CB9089590912C0177
:100CF00080912B01981749F0E92FFF27EF5BFD4FFB
:100D000080818CB99F5F90932C010895DC01309114
:100D10002B01262F932F8D91E92FFF27EF5BFD4F9E
:100D2000808321509F5F2223B1F7360F30932B0130
:100D30000895FF920F931F93CF93DF93082F80386E
:100D400011F510913A01C0E0D0E0EC2FFF27E75CED
:100D5000FE4F8281E82FFF27A5E0EE0FFF1FAA9527
:100D6000E1F7E05AFF4F82819381892B41F0CF0157
:100D70004BDB003819F40C2F005501C00F601150E7
:100D80002196112311F780912D0190912E01891B3D
:100D900087FF0BC080912B01E82FFF27EF5BFD4FF2
:100DA00091E190838F5F80932B0180912B01E82F3D
:100DB000FF27EF5BFD4F00838F5F80932B018FE058
:100DC0006822DF91CF911F910F91FF9008951F939B
:100DD000FC01162F82819381009771F01816190675
:100DE0002CF4CF01D0DA882339F004C0CF01A1DA86
:100DF000882311F0812F9DDF1F910895682F67FED2
:100E000013C080913A01681778F4E62FFF27E75C5A
:100E1000FE4F82819927B5E0880F991FBA95E1F7B7
:100E20006053805A9F4FD3DF08959927982F8827C2
:100E3000805890409093290180932801A89A0895A2
:100E400033B380B3309536953695369537708095A7
:100E5000880F8873382B832F992780729070892B85
:100E600011F080E13827222D207F832F9927807F62
:100E70009070821B9109880F991F880F991F859583
:100E800085953F70230F820F99270895D9DF982FFA
:100E9000222D82258F70292E907F207F921B892BF7
:100EA00099270895189522B708B600FE02C02FEFC3
:100EB00006C080912001281710F420932001809112
:100EC0002101821710F42093210180912201909139
:100ED0002301AC01420F511D9A0144275527542F7D
:100EE000432F322F2227AA27BB27281B390B4A0B57
:100EF0005B0B232F342F452F552747FD5A953093F1
:100F000023012093220188B7882329F478948895B7
:100F1000F89480E182BF81E088BF80913601882308
:100F200019F081E391E0B3D8C3D908950F931F93CB
:100F3000CF93DF93EC01142F022F242F3327402F60
:100F40005527C901840F951F81970CF046C0CE012B
:100F5000820F931F7DD5010F1A3028F40A3028F034
:100F6000CE013FDB02C01C3020F40B3010F0CE016C
:100F700088DB1C86013188F188899989AA89BB8917
:100F800082509040A040B0488D5F9F4FAF4FBF4F01
:100F900008F4188A8C899D89AE89BF898250904057
:100FA000A040B0488D5F9F4FAF4FBF4F08F41C8AE1
:100FB0002C893D894E895F8988899989AA89BB894D
:100FC000281739074A075B0744F48C8B9D8BAE8B3F
:100FD000BF8B288B398B4A8B5B8BDF91CF911F9115
:100FE0000F9108958F929F92AF92BF92CF92DF920E
:100FF000EF92FF920F931F93CF93DF93CDB7DEB79E
:1010000024970FB6F894DEBF0FBECDBF8C017B01D5
:10101000942E88E1841708F4A2C0442309F49FC0E9
:10102000F801A484B584C684D784F1E0F41738F4B9
:10103000242F21506F5F7F4F49E0C80177DFF70110
:101040008080E82CFF24E7FCF0948E2D807F09F04F
:1010500086C0C701877090700597E1F5F80180851B
:1010600085FF02C0C801A9DBF801248535854685C6
:10107000578529833A834B835C83808180FD04C03C
:10108000A480B580C680D7802A0D3B1D4C1D5D1DF8
:1010900029833A834B835C830FB603FE11C00FB6DE
:1010A00002FE05C08FEF9FEFAFEFBFE704C081E006
:1010B00090E0A0E0B0E889839A83AB83BC8301C051
:1010C000198289819A81AB81BC81F80184879587D7
:1010D000A687B787E0FE27C0F801808585FD23C07D
:1010E000208931894289538984859585A685B7856C
:1010F00082179307A407B50724F42487358746870A
:101100005787F801248935894689578984859585CB
:10111000A685B785281739074A075B0724F4248773
:10112000358746875787E1FE14C0F7E0F91540F090
:10113000F801808588258295880F807E805802C0BE
:10114000F801878587FD02C081E001C08FEFF801BB
:101150008787FBEF8F22F80180818829808324967E
:101160000FB6F894DEBF0FBECDBFDF91CF911F91B8
:101170000F91FF90EF90DF90CF90BF90AF909F9036
:101180008F9008955F9BD7C13CB1462D4F7E642E52
:1011900045FF1BC05C9B02C081EA0FC080912D01FE
:1011A000E82FFF27EF5BFE4F30838F5F80932D0189
:1011B00090912E01891719F482EABBDD0895303829
:1011C00009F0B9C18FED68220895252D552009F445
:1011D000C3C0E52DFF27E75CFE4F308353942150B9
:1011E00080913A01281709F0A6C190913901A92FE1
:1011F000BB27A770B07065E0AA0FBB1F6A95E1F727
:10120000A05ABF4F892F8058863040F4293130F4DE
:10121000422F6BE371E0CD01E5DE9CC0892F885839
:10122000863030F4293120F448E06BE371E031C0BE
:10123000892F8E58823060F42150263008F08AC001
:1012400050E2652E642A10922E0110922D0182C068
:10125000892F8059863090F4223081F480913B01AF
:1012600060913C01282F3327C901860F911D81977A
:1012700008F070C0CD01820F931F37C0892F8859A5
:10128000863050F4223040F0215040913B016CE315
:1012900071E0CD014BDE5EC0903A09F042C02430CF
:1012A00009F058C0E0913B01F0913C0180913D0173
:1012B00060913E01662309F44DC087FD13C09F0174
:1012C00040912B01562F942FF9018491E92FFF278C
:1012D000EF5BFD4F80832F5F3F4F51509F5F552342
:1012E00099F71BC0803819F4CF0110DD33C0E199A4
:1012F00031C09F0140912B01562F942F3FBB2EBB35
:10130000E09A8DB3E92FFF27EF5BFD4F80832F5FBE
:101310003F4F51509F5F552389F7460F40932B0154
:1013200019C0913AB9F42430A8F080913B01909112
:101330003C0130913D01303841F4422F5527435054
:1013400050406EE371E084D305C0313819F483E076
:1013500080932A0155240895832F8154863050F4B8
:10136000992745E0880F991F4A95E1F768E0805A70
:101370009F4F0FC0333241F480912B01E82FFF279C
:10138000EF5BFD4F3083C9C0343229F464E084E25E
:1013900091E0BCDC0895353251F464E080E291E0E4
:1013A000B5DC8FEF80932001109221010895363231
:1013B00019F430E1632E74C03F33B9F480912B01EE
:1013C000E82FFF27EF5BFD4F93E590838F5FE82FBA
:1013D000FF27EF5BFD4F9DE490838F5FE82FFF2792
:1013E000EF5BFD4F92E3908398C0832F805388304A
:1013F00038F4382E863010F4A9980895A99A0895E3
:101400003B3211F461E003C03D3219F46FEF80E02C
:1014100025C03034D1F480912B01E82FFF27EF5BFA
:10142000FD4F30828F5FE82FFF27EF5BFD4F10826B
:101430008F5FE82FFF27EF5BFD4F10828F5FE82F54
:10144000FF27EF5BFD4F408368C0313619F461E040
:1014500081E604C0323621F46FEF82E6CDDB0895D9
:10146000333611F432DC0895832F8451863058F4DA
:10147000832F992725E0880F991F2A95E1F780523D
:101480009240C2D70895343629F44095427091E0D5
:10149000692E06C0353631F44095427085E0682EDD
:1014A000642A0895363611F46ED80895832F8E5627
:1014B000863058F4832F9927B5E0880F991FBA9585
:1014C000E1F780569D401CD80895343711F454D666
:1014D0000895832F8557863068F4E32FFF27A5E012
:1014E000EE0FFF1FAA95E1F7E054FE4080858D7F47
:1014F000808708953E37A9F4F4E67F2E10922901E3
:101500001092280185B391E0892785BB80912B013A
:10151000E82FFF27EF5BFD4F20828F5F80932B0129
:10152000089537FF08C03093390110922A0147FD12
:1015300002C0E1E05E2E0895B6DC24DEB4DCCEDB32
:1015400008950F931F938C0146E050E06FEF70E019
:1015500088D28FE0F80184831F910F910895FF9244
:101560000F931F93CF93DF9381B7809330019FEF49
:1015700091BF22E023BF31E039BF80E885BF90935F
:10158000200185EF88BB8CE385BB8CEF82BB8AE2B0
:1015900087BB83E084BB21BB80E58DB93EB981E385
:1015A00091E0CFDF81E391E072D5F9D8552477241B
:1015B000442466243324222443DC282E80E490E053
:1015C000909338018093370188E189B91BB88AB9B3
:1015D0006ADC80E690E02DD981DB65DC80E890E074
:1015E00028D9D0DD60DC80EA90E023D977DB5BDCB2
:1015F00080EC90E01ED9C6DD56DC80EE90E019D973
:101600006DDB51DC80E091E014D9BCDD4CDC3EDCCC
:10161000772009F068C0C82FDD27CE018F71907048
:10162000892B09F460C0222D3327CE018223932316
:1016300083FF17C022FF0BC0862D962D9F5F9F70E2
:10164000807F892B682E80FD0CC0F1D60AC0832DC7
:101650008F5F382E833008F03324A998832D8F5F55
:10166000E4DB222D3327CE018223932382FF0DC09A
:1016700023FD0BC0832D33948250833010F083E020
:10168000382EA998832D8250D0DBC1FD1EDB222D80
:101690003327CE018223932380FF17C0C901809591
:1016A00090958F709070892B09F488DA21FF02C021
:1016B0008AD70BC0832D33948550823010F006E01A
:1016C000302EA99A832D8550B0DBC4FF0CC0C5FF16
:1016D00002C06FEF01C061E0641521F4822D8270B9
:1016E0008BDA01C0462E462D64FE20C080912A016F
:1016F0008823E1F480E690E0E2E6F0E020813181A9
:10170000B096809651E080329507C1F7232B71F493
:1017100080912B01E82FFF27EF5BFD4F96E290832E
:101720008F5F80932B011FEE612E6422D7DABBDB23
:101730008091280190912901009769F00197909379
:101740002901809328018F779070892B21F485B32C
:1017500091E0892785BBAADA872D772021F0815077
:10176000782E09F4A898E19942C0F0902A01FF2050
:10177000E1F000913B0110913C01EF2DFF27E75C68
:10178000FE4F6281C80179D40F5F1F4F10933C0157
:1017900000933B019F2D9F5F90932A0180913A0116
:1017A000981729F510922A0122C0E0E6F0E008E03F
:1017B00010E0808184FF04C0005D1F4FB09613C00D
:1017C000EF012496FF246881C80157D4E1990FC026
:1017D0000F5F1F4F2196F39485E0F816A1F7055D82
:1017E0001F4FFE01779621E0E032F20710F3CADCCA
:1017F000962D65FEEDCE809139018295880F880F78
:10180000807C682E692AB4E67B2E10922901109202
:10181000280185B391E0892785BB1092240110929D
:10182000250110922601109227010CC185DE80E06F
:10183000E5DA82DE81E0E2DA7FDE82E0DFDA7CDE9A
:1018400083E0DCDA79DE84E0D9DA76DE85E0D6DAA8
:1018500073DE1CDB282F882379F090912B01E92F70
:10186000FF27EF5BFD4F2073822D8F708064822BEA
:1018700080839F5F90932B0121FE02C080EA59DA9A
:1018800015DA5ADE262D67FEDDC010913A01F09080
:101890002E0190912D019F1939F0EF2DFF27EF5B5D
:1018A000FE4F8081803861F1911760F520E030E0D3
:1018B000E22FFF27E75CFE4FE281FF27A5E0EE0F56
:1018C000FF1FAA95E1F7E05AFF4F82819381892B90
:1018D000E9F411502F5F3F4F112351F72DDE809116
:1018E0002D01992720912E01821B910920913A0107
:1018F0003327821793070CF0A5C0115079F781E8C0
:1019000018DAA0C097FF0DC093E10CC0822F80545D
:10191000F7CF83EAF5CF802F8051F2CF802F80520E
:10192000EFCF91E180912B01E82FFF27EF5BFD4F77
:1019300090838F5F80932B01C0E0D0E0A22FBB2764
:10194000A074B0700C2FEF2DFF27EF5BFE4F90813E
:101950009038F9F2492F552747FD5095EC2FFF2776
:10196000E75CFE4F8281E82FFF2775E0EE0FFF1F37
:101970007A95E1F7E05AFF4F109739F1992309F46E
:1019800046C0628173819A0157FF04C02227332722
:10199000241B350B8185992787FD90958217930726
:1019A0000CF4B9CF9B01240F351FA90137FF04C0E8
:1019B00044275527421B530B82859385841795072F
:1019C0000CF4ACCF3383228322C0828193819A01AD
:1019D000281B390BE1F037FF03C0309521953F4FAD
:1019E0008185992787FD9095821793070CF493CFF3
:1019F0009A0157FF04C022273327241B350B828509
:101A00009385821793070CF489CF53834283F39411
:101A100011502196112309F095CF809124019091C6
:101A20002501A0912601B09127010196A11DB11DAC
:101A30008093240190932501A0932601B093270160
:101A4000F0922E0167FCF2CE40D97724A898C0CD41
:101A5000FB01DC0102C001900D9241505040D8F7CB
:101A60000895DC0101C06D9341505040E0F70895A6
:101A7000629FD001739FF001829FE00DF11D649F72
:101A8000E00DF11D929FF00D839FF00D749FF00DFE
:101A9000659FF00D9927729FB00DE11DF91F639F9F
:101AA000B00DE11DF91FBD01CF0111240895FFCF35
:00000001FF
